:020000040800F2
:10000000E006002089010008910100089301000822
:100010009501000897010008990100080000000000
:100020000000000000000000000000009B0100082C
:100030009D010008000000009F010008A1010008C8
:10004000A3010008A3010008A3010008A301000800
:10005000A3010008A3010008A3010008A3010008F0
:10006000A3010008A3010008A3010008A3010008E0
:10007000A3010008A3010008A3010008A3010008D0
:10008000A3010008A3010008A3010008A3010008C0
:10009000A3010008A3010008A3010008A3010008B0
:1000A000A3010008A3010008A3010008A3010008A0
:1000B00015070008A3010008A3010008A301000818
:1000C000A3010008A3010008A3010008A301000880
:1000D000A301000825080008A3010008A3010008E7
:1000E000A3010008A3010008A301000800F002F822
:1000F00000F03AF80AA090E8000C82448344AAF188
:100100000107DA4501D100F02FF8AFF2090EBAE885
:100110000F0013F0010F18BFFB1A43F0010318473B
:10012000E80D0000080E0000103A24BF78C878C11E
:10013000FAD8520724BF30C830C144BF04680C60ED
:10014000704700000023002400250026103A28BF35
:1001500078C1FBD8520728BF30C148BF0B60704739
:100160001FB51FBD10B510BD00F06EF81146FFF7AA
:10017000F7FF00F005FE00F0A0F803B4FFF7F2FF70
:1001800003BC00F0ACFC0000094880470948004768
:10019000FEE7FEE7FEE7FEE7FEE7FEE7FEE7FEE737
:1001A000FEE7FEE704480549054A064B7047000094
:1001B000B5060008ED000008E0000020E006002081
:1001C000E0020020E0020020704700000FB4044964
:1001D00010B503AA029800F009F810BC5DF814FBF2
:1001E000100000207047704770477047074B70B58C
:1001F0000D467B4400F011F80446284600F020F834
:1002000010B14FF0FF3070BD204670BD5B0B000099
:1002100001694A1C02610878704700B58FB0CDE9CA
:1002200001310021059105497944CDE903101146BA
:10023000684600F02EF80FB000BD0000E5FFFFFF9C
:10024000007B00F080007047754600F03FF8AE4636
:1002500005006946534620F00700854618B020B5D2
:10026000FFF7A0FFBDE820404FF000064FF0000769
:100270004FF000084FF0000B21F00701AC46ACE84E
:10028000C009ACE8C009ACE8C009ACE8C0098D46BB
:1002900070472DE9F04106460024D6E90170F56863
:1002A0008046304603E04146B847641C3046A847C4
:1002B0000028F8D12046BDE8F08110B50446AFF320
:1002C00000802046BDE81040FFF757BF0048704748
:1002D0007C0000202DE9F041024600250026002088
:1002E00000230024002791F803C00CF00F0591F8BB
:1002F00003C00CF0100CBCF1000F03D091F802C049
:100300004CEA050591F800C0BCF1000F31D014682B
:1003100000202BE04FF0010C0CFA00F3B1F800C004
:100320000CEA03069E4220D183004FF00F0C0CFA1A
:1003300003F7BC4305FA03FC4CEA040491F803C03C
:10034000BCF1280F06D14FF0010C0CFA00FCC2F8EA
:1003500014C00AE091F803C0BCF1480F05D14FF07A
:10036000010C0CFA00FCC2F810C0401C0828D1D3C4
:100370001460B1F800C0BCF1FF0F34DD54680020F8
:100380002EE000F1080C4FF0010808FA0CF3B1F868
:1003900000C00CEA03069E4221D183004FF00F0CEF
:1003A0000CFA03F7BC4305FA03FC4CEA040491F889
:1003B00003C0BCF1280F05D100F1080C08FA0CF8B5
:1003C000C2F8148091F803C0BCF1480F07D100F1C6
:1003D000080C4FF0010808FA0CF8C2F81080401C15
:1003E0000828CED35460BDE8F081416170470161B7
:1003F0007047000070B5002100230F22C47804B3B9
:10040000154C246804F4E064C4F5E064210AC1F1E9
:100410000403CA40447804FA03F184781440214369
:1004200009010E4C0678A155047804F01F0501243B
:10043000AC4005786D11AD0005F1E025C5F800412F
:1004400009E0047804F01F050124AC40044D06784F
:10045000761145F8264070BD0CED00E000E400E0A8
:1004600080E100E002490143024A11607047000048
:100470000000FA050CED00E029B1064AD2690243FA
:10048000044BDA6104E0034AD2698243014BDA612A
:10049000704700000010024029B1064A1269024369
:1004A000044B1A6104E0034A12698243014B1A614A
:1004B000704700000010024029B1064A92690243C9
:1004C000044B9A6104E0034A92698243014B9A61AA
:1004D000704700000010024029B1064AD26802436A
:1004E000044BDA6004E0034AD2688243014BDA60CD
:1004F000704700000010024030B5002100220024A7
:1005000000232D4D6D6805F00C0121B1042905D0A3
:10051000082923D105E0294D056022E0274D05601B
:100520001FE0254D6D6805F47012234D6D6805F4CC
:100530008034022505EB92421CB9214D55430560DC
:100540000BE01D4D6D6805F400351DB11C4D554384
:10055000056002E0194D5543056002E0174D056046
:1005600000BF00BF144D6D6805F0F0010909154D7D
:100570006B5C0568DD4045600F4D6D6805F4E0611A
:10058000090A104D6B5C4568DD4085600A4D6D6859
:1005900005F46051C90A0B4D6B5C4568DD40C560D0
:1005A000054D6D6805F44041890B074D6B5CC568CE
:1005B000B5FBF3F5056130BD0010024000127A0072
:1005C00000093D00140000202400002010B500F0B8
:1005D00001F810BD0CB50020019000903348006870
:1005E00040F480303149086000BF3048006800F4B2
:1005F000003000900198401C0190009818B90198B3
:10060000B0F5A06FF1D12948006800F4003010B1B6
:100610000120009001E0002000900098012843D1C3
:100620002348006840F0100021490860084600682F
:1006300020F0070008600846006840F002000860EB
:100640001A484068194948600846406848600846AA
:10065000406840F4806048600846406820F47C10A0
:1006600048600846406840F4E81048600846006862
:1006700040F08070086000BF0C48006800F0007017
:100680000028F9D00948406820F003000749486075
:100690000846406840F00200486000BF03484068D8
:1006A00000F00C000828F9D10CBD00000010024039
:1006B0000020024010B51348006840F001001149C5
:1006C000086008464068104908400E4948600846DE
:1006D00000680E4908400B4908600846006820F48D
:1006E000802008600846406820F4FE0048604FF40F
:1006F0001F008860FFF76AFF4FF000600449086040
:1007000010BD0000001002400000FFF8FFFFF6FEE1
:1007100008ED00E010B50121880700F017F828B1B6
:100720000121880700F003F800F0E6FB10BDCA4382
:100730000282704721B1028842F00102028004E087
:1007400002884FF6FE731A400280704730B50246A9
:10075000002000230024158A05EA0103958905EA93
:10076000010413B10CB1012000E0002030BD1AB12A
:1007700083890B43838102E083898B4383817047A4
:10078000002202881D4B98420ED01D4B98420BD080
:10079000B0F1804F08D01B4B984205D01A4B9842BD
:1007A00002D01A4B984204D14FF68F731A404B88EF
:1007B0001A43174B984207D0164B984204D04FF675
:1007C000FF431A40CB881A4302808B8883850B88AD
:1007D00003850A4B98420BD0094B984208D00E4B28
:1007E000984205D00D4B984202D00D4B984201D152
:1007F0000B7A03860123838270470000002C01409E
:10080000003401400004004000080040000C00409B
:10081000001000400014004000400140004401402E
:100820000048014010B540F226610E4800F093F8F0
:1008300020B140F226610B4800F016F840F2255135
:10084000084800F088F858B140F22551054800F0FA
:100850000BF8044800F03AF9C4B2204600F038FB27
:1008600010BD00000038014010B50022002340F602
:100870006A14A14200D100BF0A1201249440A3B21D
:10088000DC43048010BD21B1828942F40052828190
:1008900004E082894DF6FF731A40828170470000A0
:1008A00010B504462048844209D101218803FFF78E
:1008B00013FE00214FF48040FFF70EFE32E01B488C
:1008C000844209D101214804FFF7E6FD00214FF4DD
:1008D0000030FFF7E1FD25E01548844209D10121F0
:1008E0008804FFF7D9FD00214FF48020FFF7D4FDE5
:1008F00018E01048844209D10121C804FFF7CCFD5B
:1009000000214FF40020FFF7C7FD0BE00A488442A6
:1009100008D101210805FFF7BFFD00214FF4801029
:10092000FFF7BAFD10BD0000003801400044004050
:1009300000480040004C00400050004002460020AB
:10094000B1F5007F00D100BF13880B400BB101202F
:1009500000E00020704770B5024600240023002507
:10096000002040F66A16B14200D100BFC1F3421523
:1009700001F01F03012606FA03F3012D02D1968927
:10098000334006E0022D02D1168A334001E0968AF8
:1009900033400C12012606FA04F41688344013B1D1
:1009A0000CB1012000E0002070BDF0B5034600242A
:1009B00000260025002040F66A17B94200D100BF8A
:1009C0001846C1F3421401F01F06012707FA06F585
:1009D000012C01D10C3004E0022C01D1103000E0D8
:1009E00014301AB107682F43076002E00768AF436D
:1009F0000760F0BD2DE9F04786B005460E4600249D
:100A0000A24600BFA1460027B08900B100BF2F4613
:100A10002C8A4CF6FF700440F08804432C82AC8989
:100A20004EF6F3100440B0883189084371890843B9
:100A30000443AC81AC8A4FF6FF400440B0890443C4
:100A4000AC8201A8FFF758FD1F48874202D1DDF8AC
:100A500010A001E0DDF80CA0A88900F4004040B12E
:100A60000AEBCA0000EB0A1031684900B0FBF1F84C
:100A700007E00AEBCA0000EB0A1031688900B0FBFE
:100A8000F1F86420B8FBF0F004012009642101FBB7
:100A90001089A88900F4004040B1322000EBC90061
:100AA000B0FBF1F000F00700044308E0322000EB57
:100AB00009106421B0FBF1F000F00F0004432C8119
:100AC00006B0BDE8F0870000003801400146888884
:100AD000C0F308007047C1F30802828070470146E6
:100AE00000BF7047002001490870704700000020D7
:100AF00001480078704700000000002010B588B061
:100B0000FFF7F6FF002804DDFFF7ECFF0020444963
:100B100008704348007820B101282AD002287BD1F0
:100B200052E00021684600F037F99DE80F001C46AE
:100B3000CDE90623CDE90401A0470121684600F074
:100B40002BF99DE80F001C46CDE90623CDE90401F1
:100B5000A04700F00FF933490968401AB0F5FA7F51
:100B600006D901202E49087000F004F92D490860CB
:100B700052E00021684600F00FF99DE80F0014468E
:100B8000CDE90623CDE90401A0470121684600F024
:100B900003F99DE80F001C46CDE90623CDE90401C9
:100BA000A04700F0E7F81F490968401AB0F5FA7F3E
:100BB00009D902201A49087000F0DCF819490860C8
:100BC00019A0FFF703FB27E00021684600F0E4F8D6
:100BD0009DE80F001C46CDE90623CDE90401A0479E
:100BE0000121684600F0D8F89DE80F001446CDE9D1
:100BF0000623CDE90401A04700F0BCF809490968C3
:100C0000401AB0F5FA7F06D901200549087000F0B6
:100C1000B1F80449086000BF00BF08B010BD000073
:100C200001000020040000203132330A00000000DF
:100C300010B500F034F84FF4E13000F035F810BD95
:100C40001FB501210846FFF717FC4FF47A70ADF885
:100C500008004720ADF804000020ADF80A00ADF808
:100C6000060001A94FF08040FFF78AFD01221146DE
:100C70009007FFF77CFD1C208DF8000000208DF808
:100C8000010003208DF8020001208DF80300684662
:100C9000FFF7B0FB01218807FFF74CFD1FBD10B522
:100CA000FFF7CEFF10BD000010B586B0044601214D
:100CB00044F20400FFF700FC2348FFF7F1FD4FF476
:100CC0000070ADF8140003208DF8160018208DF880
:100CD000170005A91D48FFF7FDFA4FF48060ADF835
:100CE000140004208DF8170005A91848FFF7F2FA40
:100CF00001940020ADF80800ADF80A00ADF80C0032
:100D0000ADF810000C20ADF80E0001A90E48FFF759
:100D100071FE25208DF8000003208DF801008DF86C
:100D2000020001208DF803006846FFF763FB0122F3
:100D300040F225510448FFF738FE01210248FFF731
:100D4000A2FD06B010BD00000038014000080140BF
:100D500070B504460D4600BF40210548FFF7EEFD83
:100D60000028F9D0E1B20248FFF7B5FE204670BD79
:100D70000038014001480068704700000C00002066
:100D80004FF4A060FFF76EFBFFF752FF00F072F820
:100D900001E0FFF7B3FEFCE730B5022906DA044AAA
:100DA00002EB01153CCD80E83C0030BD00BFFEE702
:100DB0002800002008B501211020FFF77DFB4FF42B
:100DC0000050ADF8000010208DF8030003208DF8CE
:100DD000020069460448FFF77DFA4FF400510248CB
:100DE000FFF705FB08BD00000010014010B54FF4EF
:100DF00000510248FFF7F9FA10BD00000010014051
:100E000010B54FF400510248FFF7F1FA10BD000091
:100E10000010014008B501211020FFF74DFB4FF4F1
:100E20008040ADF8000010208DF8030003208DF8FD
:100E3000020069460448FFF74DFA4FF4804102482A
:100E4000FFF7D5FA08BD00000010014010B54FF4BF
:100E500080410248FFF7C9FA10BD000000100140B0
:100E600010B54FF480410248FFF7C1FA10BD0000F1
:100E70000010014010B500200E4908700E4848606F
:100E80000E4888600E48C860012008740D49094862
:100E900041610D4981610D49C161002406E00549A8
:100EA00001EB041148688047601CC4B2022CF6DBD9
:100EB00010BD000028000020B50D0008010E00083C
:100EC000ED0D0008150E0008610E00084D0E00081B
:100ED0000749084A1288885406490988491C322261
:100EE000B1FBF2F302FB1311024A118070470000BC
:100EF000480000200800002002480068401C01490A
:100F0000086070470C000020280F00080000002037
:100F10002800000028010008500F000828000020C9
:100F2000B8060000440100080000000000000000B6
:100F300000000000000000000000000000000000B1
:100F4000010203040102030406070809020406085B
:04000005080000ED02
:00000001FF
